:020000040800F2
:10000000482B00200101000819120008A511000862
:1000100015120008DD0E00083F2500080000000052
:10002000000000000000000000000000D51A0008D9
:10003000851000080000000047190008E91B0008AF
:100040001701000817010008170100081701000830
:100050001701000817010008170100081701000820
:100060001701000817010008170100081701000810
:100070001701000817010008170100081701000800
:1000800017010008170100081701000817010008F0
:1000900017010008170100081701000817010008E0
:1000A00017010008170100081701000817010008D0
:1000B0004D1C0008011D0008BD1F000817010008A5
:1000C00017010008170100081701000817010008B0
:1000D0001701000817010008652200081701000831
:1000E000170100081701000817010008DFF80CD0FD
:1000F00000F0FCFA00480047E12F0008482B0020E0
:1001000005480047FEE7FEE7FEE7FEE7FEE7FEE7FD
:10011000FEE7FEE7FEE7FEE7ED00000830B5054626
:100120002A460B4612F8010B13F8014B08B1A04206
:10013000F8D01CB1002802D06D1CF1E7284630BD74
:10014000421C10F8011B0029FBD1801A70470EB524
:1001500040F2334102910021CDE900110A460B46DD
:1001600000F0BEF803B000BD00F0004230F00040E7
:100170000AD0C10D01F56071C0F3160042EA0151C9
:10018000C20840071143704700200146704701F044
:10019000004330B421F0004150EA010206D00A0DBC
:1001A000A2F56072C1F31301002A02DC30BC00200A
:1001B0007047440F44EAC104C100E01830BC00EBB2
:1001C000C25000F047B830B50B460146002020224F
:1001D000012409E021FA02F59D4205D303FA02F554
:1001E000491B04FA02F52844151EA2F10102F1DCB4
:1001F00030BD2DE9F05F0546002092469B468846BB
:100200000646814640241BE0284641464746224692
:1002100000F08DFA53465A46C01A914110D3114648
:100220001846224600F074FA2D1A67EB01084F4673
:1002300022460120002100F06BFA17EB00094E4125
:10024000201EA4F10104DFDC484631462A4643461D
:10025000BDE8F09F0029A8BF7047401C490008BFB7
:1002600020F00100704710B4B0FA80FC00FA0CF0E6
:1002700050EA010404BF10BC704749B1CCF120041E
:1002800021FA04F411FA0CF118BF012121430843AB
:10029000A3EB0C01CB1D4FEA00614FEA102042BFD7
:1002A000002010BC704700EBC35010440029A4BFCD
:1002B00010BC7047401C490008BF20F0010010BC72
:1002C000704710B5141E73F1000408DA401C41F1A8
:1002D000000192185B411A4301D120F0010010BDCA
:1002E0002DE9F04D92469B4611B1B1FA81F202E040
:1002F000B0FA80F22032904600F00AFA04460F4627
:1003000040EA0A0041EA0B0153465A46084313D01B
:10031000114653EA010019D0C8F14002504600F0DE
:1003200006FA05460E4650465946424600F0F0F998
:10033000084305D0012004E020463946BDE8F08D91
:100340000020054346EAE0762C4337430A986305CC
:10035000E40AA0EB08000022FD0A44EA47540A30F0
:1003600002D500200146E9E7010510196941DDE9E0
:10037000084500196941BDE8F04DA2E72DE9FE4F9F
:10038000804681EA0300C00F0C46009021F0004136
:1003900023F00045B8EB0200A94105D240462146B2
:1003A00090461C460B46024623F00040104347D0BF
:1003B000270DC7F30A00C3F30A510290401A0190B7
:1003C00040286BDAC3F3130040F4801B0098924678
:1003D00020B10023D2EB030A63EB0B0B01985946C3
:1003E000C0F14002504600F093F906460D465046D3
:1003F0005946019A00F0ABF910EB08006141002466
:1004000087EA115284EAE7731A4340D0009A62B334
:10041000019A012A4FEA075215DC001B61EB020129
:100420004FF0004202EA0752CDE90042001C41F5BC
:10043000801132462B46FFF753FF03B0BDE8F08F23
:1004400040462146F9E7001B61EB0201001C41F523
:10045000801300185B412018A2F5001747EB030139
:1004600040EAD570B6196D4111E06D084FEA3606C5
:1004700045EAC0754FEA0752001B61EB0201001C00
:1004800041F5801149084FEA3000001951413246C8
:100490002B4603B0BDE8F04FFFF713BF00980122D1
:1004A00040000023D0EB020263EBE073009821468A
:1004B0004FEAE074B8EB000061EB0401E9E783F078
:1004C00000435BE781F0004158E72DE9FE4F81EAE8
:1004D000030404F0004421F0004100944FF0000BAD
:1004E00023F0004350EA01045ED052EA03045BD0DB
:1004F000C3F30A54C1F30A552C44A4F2F334019413
:10050000A0FB0254C1F3130141F48011C3F31303A0
:1005100043F4801301FB024400FB034E840A970A54
:1005200044EA815447EA8357A4FB076802958D0A81
:1005300005FB07854FEA932C04FB0C542705029D0D
:100540004FEA065847EA1637B5EB08056EEB070C7D
:10055000870E920E47EA811742EA8312A7FB020137
:10056000B6EB0B0164EB00042B0D43EA0C335E1871
:1005700044EB1C50DA465146E7FB0201C5F3130475
:100580004FEA0B3343EA14534FEA0432019C43EA27
:100590000603A4F10C040294009CCDE900B4FFF71B
:1005A0009FFE03B0BDE8F08F00200146F9E72DE97A
:1005B000F04D81EA030404F0004B21F0004514469D
:1005C0004FF0000A23F0004150EA050220D054EA1F
:1005D00001021DD0C5F30A570246C5F31303C1F348
:1005E0001300C1F30A5640F4801543F48013A7EBBF
:1005F0000608101BD64608F2FD3873EB050002D33F
:1006000008F1010801E092185B41B8F1000F03DA2C
:1006100000200146BDE8F08D00204FF48011064611
:1006200084460EE0171B73EB050705D3121B63EB23
:10063000050306434CEA010C49084FEA30009218C2
:100640005B4150EA0107EDD152EA030012D082EA81
:10065000040083EA0501084305D0101BAB4106D214
:100660000122002306E000224FF0004302E06FF079
:10067000010253101AEB06004CEB085110EB0A0074
:1006800041EB0B01BDE8F04DFFF71BBEC1F30A5271
:10069000C1F3130140F2FF3341F480119A4202DAB0
:1006A00000200146704740F233439A42A2F233429F
:1006B00002DC524200F03BB800F02AB830B5041E0C
:1006C00071F1000404DB4FF00044404264EB01018F
:1006D000141E73F1000405DB1C464FF00043524228
:1006E00063EB0403994208BF904230BD064C074DAE
:1006F00006E0E06840F0010394E8070098471034F2
:10070000AC42F6D3FFF7F6FC345000085450000812
:10071000202A04DB203A00FA02F1002070479140C1
:10072000C2F1200320FA03F3194390407047202AB6
:1007300004DB203A21FA02F00021704721FA02F38B
:10074000D040C2F120029140084319467047202A48
:1007500006DBCB17203A41FA02F043EAE07306E0E9
:1007600041FA02F3D040C2F12002914008431946F9
:10077000704721B1826842F00102826003E0826822
:1007800022F001028260704710B50446124884428C
:1007900008D10121401501F023F90021601501F075
:1007A0001FF917E00D48844208D10121001501F01E
:1007B00017F90021201501F013F90BE008488442D5
:1007C00008D10121C80301F00BF900214FF40040CA
:1007D00001F006F910BD000000240140002801408E
:1007E000003C014021B1826842F48012826003E043
:1007F000826822F4801282607047014600208A6875
:1008000002F004020AB1012000E000207047014616
:10081000C86C80B27047014600208A6802F0080266
:100820000AB1012000E000207047000030B5024608
:100830000020002350680F4C20400D790C6844EADA
:1008400005242043506090680B4C2040D1E90254AD
:100850002C434D7944EA450420439060D06A20F44B
:1008600070000C7C641EE4B2234340EA0350D06263
:1008700030BD0000FFFEF0FFFDF7F1FFF0B50446CC
:100880000D4600200021092D11DDE068A5F10A06C2
:1008900006EB4607072606FA07F18843A5F10A0684
:1008A00006EB460603FA06F10843E0600CE0206917
:1008B00005EB4507072606FA07F1884305EB4506D1
:1008C00003FA06F108432061072A0FDA606B561E0F
:1008D00006EB86071F2606FA07F18843561E06EB2D
:1008E000860605FA06F10843606322E00D2A0FDA56
:1008F000206BD61F06EB86071F2606FA07F18843F2
:10090000D61F06EB860605FA06F10843206310E0C1
:10091000E06AA2F10D0606EB86071F2606FA07F12C
:100920008843A2F10D0606EB860605FA06F1084398
:10093000E062F0BD816841F0080181607047816824
:1009400041F004018160704700B587B001214FF488
:10095000017001F035F84FF4004000F0F5FF012080
:10096000ADF8040000208DF8070001A91C4800F034
:100970008AFB1C48FFF708FF002002908DF80C004E
:100980008DF80D004FF40020049000200590012008
:100990008DF8180002A91348FFF748FF01211148FC
:1009A000FFF720FF0723012200210E48FFF766FF13
:1009B00001210C48FFF7DDFE0A48FFF7BBFF00BF2F
:1009C0000848FFF728FF0028FAD10648FFF7B7FFCD
:1009D00000BF0448FFF711FF0028FAD107B000BD9F
:1009E000000801400024014010B500F003F800F0B9
:1009F000B7F810BD08B50121042000F0E1FF4FF465
:100A00000060ADF8000010208DF8030003208DF881
:100A1000020069460B4800F036FB01200A490860D5
:100A20001020ADF8000028208DF8030003208DF879
:100A300002006946034800F026FB4FF4E13002F063
:100A4000ADFB08BD00080140AC0121422DE9F04199
:100A500004460D46002620462946FFF798FB074628
:100A600000F066F800F03AF80F48006868B1012617
:100A70000E480078B0B901200C49087000200C49DC
:100A800008700CA001F05EFD0CE00026084800781C
:100A900040B90120064908700020044908700AA0E6
:100AA00001F050FDBDE8F08110012142000000205E
:100AB000010000200D0A626C6520636F6E6E656335
:100AC00074210D0A000000000D0A626C6520646943
:100AD00073636F6E6E656374210D0A0070B5002438
:100AE00000251048008800F40040D0B10D4800886F
:100AF000C0F30E0500200C4948550A49088000BF84
:100B00000DE000BF4021094801F048FC0028F9D061
:100B10000548015D054801F00EFD601C84B2AC4241
:100B2000EFDB70BD020000201025002000380140DE
:100B300070B504462046FFF717FB05462A460B46CC
:100B400001A002F00BFB70BD57616E6752656E6AC3
:100B500069653A20252E31662E62706D0000000016
:100B60001CB500206C4908600FE00A226BA16DA043
:100B700002F0A6F900B90FE06C480068C0436C4968
:100B8000C1F88801642002F0FBF9052269A165A083
:100B900002F096F90028E8D100BF052267A168A0FD
:100BA00002F08EF910B967A001F0CCFC67A269A130
:100BB0006B4801F0D7FC0A2260A1694802F080F975
:100BC00020B9674967A001F0BDFC03E0644968A053
:100BD00001F0B8FC69A26CA1614801F0C3FC0A22D3
:100BE00056A15F4802F06CF920B95D495DA001F0A3
:100BF000A9FC03E05A495EA001F0A4FC062265A10D
:100C0000574801F0AFFC0A224CA1554802F058F9B0
:100C100020B9534953A001F095FC03E0504954A07A
:100C200001F090FC0120002108234FF4E132CDE9CE
:100C300000105BA14A4801F095FC0A223FA14848F8
:100C400002F03EF920B9464946A001F07BFC03E0E2
:100C5000434947A001F076FC052256A1404801F027
:100C600081FC0A2235A13E4802F02AF920B93C490C
:100C70003CA001F067FC03E039493DA001F062FCB3
:100C80000A222EA14FA002F01BF918B952A001F0C0
:100C900059FC02E056A001F055FC0A2227A15BA0F6
:100CA00002F00EF918B95CA001F04CFC02E05FA064
:100CB00001F048FC0A2221A162A002F001F918B952
:100CC00065A001F03FFC02E06AA001F03BFC0A22B3
:100CD0001AA170A002F0F4F818B972A001F032FC69
:100CE00002E075A001F02EFC532279A11C4801F00E
:100CF00039FC0A2211A11A4802F0E2F820B9184979
:100D000018A001F01FFC03E0154919A001F01AFC1E
:100D10000120014908601CBDA00121424552524FEB
:100D2000520000002B2B2B61000000008881224222
:100D300000802242612B6F6B000000004F4B0000CF
:100D4000415400004154204F4B0D0A0041544B2D9B
:100D500057524A0041542B4E414D453D25730000EA
:100D6000D8040020257320204F4B0D0A00000000FE
:100D7000257320204552524F520D0A0041544B2DED
:100D800057524A303100000041542B48454C4C4FDB
:100D90003D25730041542B54504C3D256400000008
:100DA00041542B554152543D25642C25642C256417
:100DB0002C25640041542B41445054494D3D256439
:100DC0000000000041542B4C494E4B5041535345B9
:100DD0004E3D4F464600000041542B4C494E4B506F
:100DE000415353454E3D4F464620204F4B0D0A0080
:100DF00041542B4C494E4B50415353454E3D4F4669
:100E00004620204552524F520D0A000041542B4CAF
:100E10004544454E3D4F4E0041542B4C4544454EB4
:100E20003D4F4E20204F4B0D0A00000041542B4CEB
:100E30004544454E3D4F4E20204552524F520D0ADB
:100E40000000000041542B534C415645534C45453E
:100E500050454E3D4F46460041542B534C4156455C
:100E6000534C454550454E3D4F464620204F4B0D77
:100E70000A00000041542B534C415645534C454504
:100E800050454E3D4F464620204552524F520D0A86
:100E90000000000041542B4D41585055543D4F46E1
:100EA0004600000041542B4D41585055543D4F468B
:100EB0004620204F4B0D0A0041542B4D41585055B0
:100EC000543D4F464620204552524F520D0A0000D5
:100ED00041542B4D4F44453D2563000000BFFEE7C4
:100EE00021B1026842F00102026004E002684FF69C
:100EF000FE731A400260704701684FF6FE7211409F
:100F000001600021016041608160C1604B498842FD
:100F100008D14A490839496841F00F01474A083A5F
:100F200051608AE045491431884208D14349083963
:100F3000496841F0F001414A083A51607DE03F497B
:100F40002831884208D13D490839496841F4706127
:100F50003A4A083A516070E038493C31884208D139
:100F600036490839496841F47041344A083A5160B9
:100F700063E032495031884208D130490839496824
:100F800041F470212D4A083A516056E02B496431F2
:100F9000884208D129490839496841F47001274A33
:100FA000083A516049E025497831884208D12349FF
:100FB0000839496841F07061204A083A51603CE0C4
:100FC0001F49884206D1011F096841F00F01021F25
:100FD000116032E01A491431884208D11849091FBA
:100FE000096841F0F001164A121F116025E014490A
:100FF0002831884208D11249091F096841F47061FB
:101000000F4A121F116018E00D493C31884208D187
:101010000B49091F096841F47041094A121F116008
:101020000BE007495031884207D10549091F09687B
:1010300041F47021024A121F1160704708000240FB
:101040000804024010B50022026847F6F0739A4384
:101050000C6A8B6823430C6923434C6923438C69D6
:101060002343CC6923434C6A23438C6A23431A43AA
:101070000260CB6843600B6883604B68C36010BD3F
:101080004160704770472DE9F04102460025002677
:10109000002000230024002791F803C00CF00F0566
:1010A00091F803C00CF0100CBCF1000F03D091F8C4
:1010B00002C04CEA050591F800C0BCF1000F31D028
:1010C000146800202BE04FF0010C0CFA00F3B1F88B
:1010D00000C00CEA03069E4220D183004FF00F0CA3
:1010E0000CFA03F7BC4305FA03FC4CEA040491F83C
:1010F00003C0BCF1280F06D14FF0010C0CFA00FC24
:10110000C2F814C00AE091F803C0BCF1480F05D141
:101110004FF0010C0CFA00FCC2F810C0401C08286B
:10112000D1D31460B1F800C0BCF1FF0F34DD5468B6
:1011300000202EE000F1080C4FF0010808FA0CF333
:10114000B1F800C00CEA03069E4221D183004FF0A3
:101150000F0C0CFA03F7BC4305FA03FC4CEA040439
:1011600091F803C0BCF1280F05D100F1080C08FA72
:101170000CF8C2F8148091F803C0BCF1480F07D1F5
:1011800000F1080C4FF0010808FA0CF8C2F81080C2
:10119000401C0828CED35460BDE8F08141617047FF
:1011A0000161704700BFFEE7032000BF011EA0F1F0
:1011B0000102D0B2FAD1704708B50121102000F029
:1011C000FFFB10208DF803004002ADF80000032063
:1011D0008DF8020069460448FFF755FF4FF40051AF
:1011E0000148FFF7DBFF08BD0010014010B54FF4C8
:1011F00000510248FFF7D4FF10BD0000001001406D
:1012000010B54FF400510248FFF7C8FF10BD0000B1
:101210000010014000BFFEE77047000070B50021DC
:1012200000230F22C47804B3154C246804F4E0644E
:10123000C4F5E064210AC1F10403CA40447804FA09
:1012400003F184781440214309010E4C0678A1551E
:10125000047804F01F050124AC4005786D11AD0041
:1012600005F1E025C5F8004109E0047804F01F0508
:101270000124AC40044D0678761145F8264070BD37
:101280000CED00E000E400E080E100E002490143F1
:10129000024A1160704700000000FA050CED00E002
:1012A00070B500240CE0002506E00020074901EBA2
:1012B000C5010855681CC5B2802DF6DB601CC4B2A0
:1012C000082CF0DB00F030F970BD00005800002061
:1012D000F0B514460B46CF1701EB5777C7F3C7029B
:1012E000CF1701EB5777FF10A1EBC707FEB2012321
:1012F000B340DDB24CB1134B03EBC0039B5C2B43FB
:10130000104F07EBC007BB541AE00E4B03EBC003B2
:101310009B5CDB430B4F07EBC007BB54094B03EB54
:10132000C0039B5C2B43074F07EBC007BB54054B27
:1013300003EBC0039B5CDB43024F07EBC007BB54CE
:10134000F0BD00005800002010B54FF400710C48AB
:10135000FFF726FF4FF480710948FFF721FFFFF7E1
:1013600023FF4FF400710648FFF718FFFFF71CFF3B
:101370004FF480710248FFF711FFFFF715FF10BD12
:10138000000C014010B54FF400710848FFF706FF4C
:101390004FF480710548FFF703FFFFF705FF4FF497
:1013A00000710248FFF7FCFE10BD0000000C014078
:1013B00010B54FF400710A48FFF7F2FEFFF7F4FE94
:1013C0004FF480710648FFF7EBFEFFF7EDFE4FF498
:1013D00080710348FFF7E2FEFFF7E6FE10BD000054
:1013E000000C014008B50121082000F0E9FA4FF493
:1013F0008070ADF8000014208DF8030003208DF8F4
:10140000020069464148FFF73EFE4FF480713F48B5
:10141000FFF7C6FE4FF40070ADF8000069463B4888
:10142000FFF731FE4FF400713848FFF7B9FEC820CE
:1014300001F0A6FD0021AE2000F069FA0021084667
:1014400000F065FA0021102000F061FA0021402030
:1014500000F05DFA0021812000F059FA0021CF2030
:1014600000F055FA0021A12000F051FA0021C82017
:1014700000F04DFA0021A62000F049FA0021A82032
:1014800000F045FA00213F2000F041FA0021D3206E
:1014900000F03DFA0021084600F039FA0021D5207D
:1014A00000F035FA0021802000F031FA0021D92027
:1014B00000F02DFA0021F12000F029FA0021DA20B5
:1014C00000F025FA0021122000F021FA0021DB2093
:1014D00000F01DFA0021302000F019FA0021202030
:1014E00000F015FA0021022000F011FA00218D20F1
:1014F00000F00DFA0021142000F009FAFFF7D0FEE9
:101500000021AF2000F003FA08BD0000000C0140EC
:1015100010B50246012000E050430B1EA1F101046A
:10152000E1B2F9D110BD000070B500242BE004F148
:10153000B001C8B2002100F0EAF90021084600F02D
:10154000E6F90021102000F0E2F9FFF7FDFE782017
:1015500000F01EF8FFF72CFF402000F019F8FFF70D
:1015600027FF002509E0094901EBC501085D00F0EE
:101570000FF8FFF71DFF681CC5B2802DF3DBFFF7E6
:1015800001FF601CC4B2082CD1DB70BD58000020E4
:1015900070B5044600251FE004F0800028B14FF428
:1015A00000710F48FFF7FCFD04E04FF400710C4898
:1015B000FFF7F4FDFFF7F8FD4FF480710848FFF7DF
:1015C000EFFDFFF7F1FD4FF480710548FFF7E6FDF1
:1015D0006006040E681CC5B2082DDDDB70BD00007E
:1015E000000C01402DE9FE4F0746884692461C46F6
:1015F0000197CDF80080082C02D14FF006091FE0BA
:101600002046E31704EB5373DB1021464FEAE47CDA
:1016100004EB5C7C4FEAEC0CA4EBCC0CBCF1000FAF
:1016200002D04FF0010C01E04FF0000C6344224661
:1016300004EBD27C4FEA6C0C03FB0CF303F0FF09C4
:10164000AAF12000C6B200255EE0082C07D106EB07
:101650004600304901EB400010F805B01DE00C2CAD
:1016600007D106EB46002C4901EB800010F805B0CD
:1016700013E0102C05D1294800EB061010F805B036
:101680000BE0182C07D106EBC600254901EB8000C2
:1016900010F805B001E0BDE8FE8F002002901CE0CC
:1016A0000BF0010028B1414638460C9AFFF710FEB6
:1016B00009E00C9808B9012000E0002002464146EC
:1016C0003846FFF705FE4FEA6B0B08F1010000F00A
:1016D000FF080298401CC0B2029002980828DFDB85
:1016E000781CC7B2082C0BD004EBD4714A100199B6
:1016F000791A8A4204D1019F00980830C0B2009044
:10170000DDF80080681CC5B24D459EDBFFF70CFF7D
:1017100000BFC0E784320008AC340008203900085C
:10172000103F00082DE9FC5F0746884616461C4618
:10173000BB46CDF804802046E21704EB5272D2106B
:101740002146E31704EB5373DB10A4EBC3030BB187
:10175000012300E000231A44624392B20092002564
:1017600055E0102C05D12D4800EB861010F805A08F
:101770001BE0182C07D106EBC600294901EBC0007D
:1017800010F805A011E0202C05D1264800EBC6106A
:1017900010F805A009E0402C05D1234800EB4620B5
:1017A00010F805A001E0BDE8FC9F4FF000091CE027
:1017B0000AF0010028B1414638460C9AFFF788FD2F
:1017C00009E00C9808B9012000E0002002464146DB
:1017D0003846FFF77DFD4FEA6A0A08F1010000F084
:1017E000FF0809F1010000F0FF09B9F1080FDFDB84
:1017F000781CC7B2A7EB0B00A04204D15F4601984A
:101800000830C0B20190DDF80480681C85B20098F1
:101810008542A6DBFFF788FE00BFC4E76C4C0008DA
:101820006C4D0008B44D0008344E00082DE9FF4F00
:1018300083B0064691461F46DDE9104A4FF0000B83
:10184000082C01D14FF0020B002532E0781B401E1E
:10185000C1B20A20FFF75CFEB9FBF0F00A21B0FB31
:10186000F1F201FB1208B8F1000F0FD104EBD471B3
:101870000BEB610101FB0561C8B223463022CDF8B4
:1018800000A002940499FFF7ADFE10E004EBD471C0
:101890000BEB610101FB0561C8B208F13001CAB26E
:1018A0002346CDF800A002940499FFF79BFE681C24
:1018B000C5B2BD42CADBFFF737FE07B0BDE8F08F07
:1018C0002DE9F84306460F4614461D46DDF82080F4
:1018D00013E0CDF8008022782B4639463046FFF7DA
:1018E00081FE082D02D1B01DC6B205E0284605EBE9
:1018F000D07106EB6101CEB2641C2078202802DB97
:1019000020787E28E5DDFFF70FFEBDE8F88370B58F
:1019100005460C46FFF718FD7820FFF739FEFFF764
:1019200047FD1CB14020FFF733FE02E00020FFF727
:101930002FFEFFF73DFD2846FFF72AFEFFF738FD93
:10194000FFF720FD70BD704701460020034A506834
:1019500020F44040084350607047000000100240EF
:1019600029B1064A52690243044B5A6104E0034A12
:1019700052698243014B5A617047000000100240D7
:1019800029B1064AD2690243044BDA6104E0034AF2
:10199000D2698243014BDA617047000000100240B7
:1019A00029B1064A12690243044B1A6104E0034A52
:1019B00012698243014B1A61704700000010024017
:1019C00029B1064A92690243044B9A6104E0034A32
:1019D00092698243014B9A617047000000100240F7
:1019E00029B1064AD2680243044BDA6004E0034A94
:1019F000D2688243014BDA60704700000010024059
:101A000030B500210022002400232D4D6D6805F023
:101A10000C0121B1042905D0082923D105E0294D65
:101A2000056022E0274D05601FE0254D6D6805F437
:101A30007012234D6D6805F48034022505EB924247
:101A40001CB9214D554305600BE01D4D6D6805F433
:101A500000351DB11C4D5543056002E0194D55433D
:101A6000056002E0174D056000BF00BF144D6D68B2
:101A700005F0F0010909154D6B5C0568DD40456016
:101A80000F4D6D6805F4E061090A104D6B5C456807
:101A9000DD4085600A4D6D6805F46051C90A0B4D43
:101AA0006B5C4568DD40C560054D6D6805F44041DF
:101AB000890B074D6B5CC568B5FBF3F5056130BD5F
:101AC0000010024000127A0000093D004000002092
:101AD00050000020704710B500F002F810BD000063
:101AE0000CB50020019000903348006840F480302D
:101AF0003149086000BF3048006800F400300090B1
:101B00000198401C0190009818B90198B0F5A06F99
:101B1000F1D12948006800F4003010B10120009094
:101B200001E0002000900098012843D1234800687C
:101B300040F01000214908600846006820F00300CA
:101B400008600846006840F0020008601A484068D3
:101B5000194948600846406848600846406840F4B3
:101B6000806048600846406820F47C104860084661
:101B7000406840F4E81048600846006840F0807013
:101B8000086000BF0C48006800F000700028F9D021
:101B90000948406820F0030007494860084640684B
:101BA00040F00200486000BF0348406800F00C00AD
:101BB0000828F9D10CBD00000010024000200240AE
:101BC000042808D14FF0E021096941F004014FF0E9
:101BD000E022116107E04FF0E021096921F00401E2
:101BE0004FF0E022116170477047000010B51348B4
:101BF000006840F00100114908600846406810493B
:101C000008400E494860084600680E4908400B49E4
:101C100008600846006820F4802008600846406894
:101C200020F4FE0048604FF41F008860FFF753FF68
:101C30004FF000600449086010BD00000010024031
:101C40000000FFF8FFFFF6FE08ED00E010B50121EF
:101C5000880700F01DFAF0B10121880700F009FAA9
:101C60000D480078002808DD0B480078401EC0B2FF
:101C70000949087008B9FFF7B9FA0848016800680F
:101C8000401C064A10600A2905D30020114608604E
:101C900001200349087010BD0A0000203C0000200C
:101CA000080000207FB505460C4601210846FFF7D5
:101CB00067FEADF80850ADF804400020ADF80A000A
:101CC000ADF8060001A94FF0804000F007FA0122AC
:101CD0001146900700F0EDF91C208DF8000001205E
:101CE0008DF8010003208DF8020001208DF803001B
:101CF0006846FFF793FA0121880700F0BDF97FBD20
:101D000070B5002401217C4800F0C2F9002875D08C
:101D10007A48FEF77CFD0646C01706EB90708010EF
:101D20007749086077480068801C76490860084653
:101D3000006875490968401A74490860704800686D
:101D400073490968884219DA72480068052190FBD6
:101D5000F1F000EB40006D49096888420EDA6848EE
:101D600000686D490968884208DAFFF749FA0120DE
:101D70006A490870624800686749086060480068FE
:101D800063490968884209DD5D480068644909685B
:101D9000884203DD5A480068614908605B48006872
:101DA000FA2863DD564800685949096888425DDDB4
:101DB0005C480078002859D156480068052190FBFE
:101DC000F1F000EB40005149096888424EDA0120E9
:101DD000544908704B4800684B490968401A4D49FE
:101DE000086048480068484908604F48007878B162
:101DF00000204D490870002400BF07E075E0454809
:101E000000684A4941F82400601CC4B2092CF6DD80
:101E10004748007830B10020454908700120424908
:101E2000087070BD002500240BE04049601C51F88B
:101E3000200041F82400084650F824000544601CA6
:101E4000C4B2082CF1DD33480068384948620846BE
:101E5000406A05440A20B5FBF0F54EF66020B0FB61
:101E6000F5F03449086001203349087024480068BF
:101E70002749096888421EDA2A48007801281AD1C1
:101E80000020284908702648006823490968401A3C
:101E90002A490860086800EBD0711F4A126802EBFB
:101EA00061011B4A1160104600681D490860104618
:101EB0000068194908601548006840F6C411884256
:101EC00013DD4FF40070124908601549086012498B
:101ED00008600C4800680C4908600120144908702B
:101EE000002011490870144908700121024800F0CF
:101EF000C0F800BF95E70000000400400024014046
:101F0000100000201C0000202000002034000020D1
:101F10002C00002014000020280000200A000020CF
:101F20002400002018000020390000202029002073
:101F3000380000200C000020190000203000002094
:101F40007FB505460C4601210220FFF719FDADF8CB
:101F50000850ADF804400020ADF80A00ADF80600C6
:101F600001A9154800F0BAF82021134800F0AAF89A
:101F70000121114800F07AF8012211460E4800F0C4
:101F800098F801210C4800F077F81D208DF800002A
:101F900000208DF801008DF8020001208DF803006B
:101FA0006846FFF73BF900210220FFF7E9FC012119
:101FB0000220FFF7E5FC7FBD0004004010B50121C1
:101FC000084800F065F860B10121064800F051F8BA
:101FD0000548008840F4004003490880002000F0D4
:101FE00031F810BD00080040020000207FB5054612
:101FF0000C4601210420FFF7C3FCADF80450ADF8F6
:1020000000400020ADF80600ADF8020069460C481B
:1020100000F064F801221146094800F04AF81E2039
:102020008DF80C0001208DF80D0002208DF80E00B7
:1020300001208DF80F0003A8FFF7F0F87FBD000026
:102040000008004010B5044644B10021064800F0E5
:1020500042F80121044800F00FF803E00021024893
:1020600000F00AF810BD000000080040CA430282D8
:102070007047CA430282704721B1028842F00102D0
:10208000028004E002884FF6FE731A400280704717
:1020900030B50246002000230024158A05EA01031A
:1020A000958905EA010413B10CB1012000E000207C
:1020B00030BD1AB183890B43838102E083898B434E
:1020C0008381704782884FF68F731A40828082889E
:1020D0000A43828070478184704700000022028892
:1020E0001D4B98420ED01D4B98420BD0B0F1804F43
:1020F00008D01B4B984205D01A4B984202D01A4B7D
:10210000984204D14FF68F731A404B881A43174BED
:10211000984207D0164B984204D04FF6FF431A401E
:10212000CB881A4302808B8883850B8803850A4BF2
:1021300098420BD0094B984208D00E4B984205D0DC
:102140000D4B984202D00D4B984201D10B7A038679
:102150000123838270470000002C014000340140BD
:102160000004004000080040000C00400010004047
:10217000001400400040014000440140004801407C
:1021800070B58CB006460C46154601210846FFF78F
:10219000E7FB3046FEF7B0FE019402951020039055
:1021A0000020049005908020069000200790089061
:1021B00009904FF480500A9000200B9001A93046FE
:1021C000FEF740FF0CB070BD70B504460D4600210F
:1021D0002046FEF785FE29462046FEF751FF0121E5
:1021E0002046FEF77DFE70BD00B585B0012144F2AA
:1021F0000400FFF7E5FB4FF40070ADF81000182065
:102200008DF8130003208DF8120004A91348FEF77F
:102210003AFF4FF48060ADF8100004208DF81300F1
:1022200004A90E48FEF72FFF4FF4E1300090002084
:10223000ADF80400ADF80600ADF80800ADF80C00EC
:102240000C20ADF80A006946054800F003F90121A9
:10225000034800F03FF805B000BD00000008014051
:102260000038014010B540F22551164800F0A3F89F
:10227000F8B1144800F05AF9C4B21348008800F4C9
:102280000040B0B910480088B0F5806F12DA002124
:102290000E48FFF720FF0C48008810B90120FFF717
:1022A000D1FE094801880088401C074A1080084870
:1022B000445405E00448008840F400400249088086
:1022C00010BD000000440040020000200008004053
:1022D0001025002021B1828942F40052828104E05D
:1022E00082894DF6FF731A40828170471AB1838A42
:1022F0000B43838202E0838A8B4383827047000012
:1023000010B504462048844209D101218803FFF713
:1023100067FB00214FF48040FFF762FB32E01B486F
:10232000844209D101214804FFF73AFB00214FF410
:102330000030FFF735FB25E01548844209D1012123
:102340008804FFF72DFB00214FF48020FFF728FBC6
:1023500018E01048844209D10121C804FFF720FB8E
:1023600000214FF40020FFF71BFB0BE00A488442DA
:1023700008D101210805FFF713FB00214FF480105D
:10238000FFF70EFB10BD0000003801400044004084
:1023900000480040004C0040005000400246002031
:1023A000B1F5007F00D100BF13880B400BB10120B5
:1023B00000E00020704770B502460024002300258D
:1023C000002040F66A16B14200D100BFC1F34215A9
:1023D00001F01F03012606FA03F3012D02D19689AD
:1023E000334006E0022D02D1168A334001E0968A7E
:1023F00033400C12012606FA04F41688344013B157
:102400000CB1012000E0002070BDF0B503460024AF
:1024100000260025002040F66A17B94200D100BF0F
:102420001846C1F3421401F01F06012707FA06F50A
:10243000012C01D10C3004E0022C01D1103000E05D
:1024400014301AB107682F43076002E00768AF43F2
:102450000760F0BD2DE9F04786B005460E46002422
:10246000A24600BFA1460027B08900B100BF2F4699
:102470002C8A4CF6FF700440F08804432C82AC890F
:102480004EF6F3100440B08831890843718908433F
:102490000443AC81AC8A4FF6FF400440B08904434A
:1024A000AC8201A8FFF7ACFA1F48874202D1DDF8E1
:1024B00010A001E0DDF80CA0A88900F4004040B1B4
:1024C0000AEBCA0000EB0A1031684900B0FBF1F8D2
:1024D00007E00AEBCA0000EB0A1031688900B0FB84
:1024E000F1F86420B8FBF0F004012009642101FB3D
:1024F0001089A88900F4004040B1322000EBC900E7
:10250000B0FBF1F000F00700044308E0322000EBDC
:1025100009106421B0FBF1F000F00F0004432C819E
:1025200006B0BDE8F0870000003801400146888809
:10253000C0F308007047C1F308028280704700BFF3
:10254000FEE700000FB4054B10B503A9044A02983A
:1025500000F000F910BC5DF814FB0000BD2F00086E
:10256000540000200FB4084B10B504A902AA039828
:1025700000F0F0F8044602A9002000F082FC20469A
:1025800010BC5DF814FB0000832E000837B514461C
:102590000846064B6A46214600F0DCF804466946C8
:1025A000002000F06EFC20463EBD0000832E000897
:1025B00002E008C8121F08C1002AFAD1704770470C
:1025C000002001E001C1121F002AFBD1704700006A
:1025D0002DE9FF5F82B00021DDE90430020DDDF856
:1025E00040B0034318D044F61050A2F2FF324243E9
:1025F0001514119801281FD0A5EB0B00401C5FEAB1
:10260000000A4FF000064E4FDFF83891B0465046B2
:1026100015D5CAF1000413E0119801244AA301283A
:1026200001D16FEA0B010298119AC0E90031C0E9AB
:10263000024206B0BDE8F09FCBF10000DFE70446A0
:102640000021404A491842EB0450CDE9001012E045
:10265000E00707D032463B4640464946FDF735FF86
:102660008046894632463B4610461946FDF72DFF07
:1026700006460F466410002CEAD1DDE90401DDE9CD
:102680000023BAF1000F06DAFDF71FFF42464B4662
:10269000FDF71BFF05E0FDF78AFF42464B46FDF7BD
:1026A00086FF04460E460022284BFEF707F803D8A3
:1026B0004FF0FF30014607E00022254B204631460F
:1026C000FDF75CFEFDF7E2FF102409E0002C0ADBB9
:1026D0000A220023FDF78DFD039B30321A55641E3C
:1026E00050EA0102F2D1641C039AC4F111031444AC
:1026F000119A012A03D0012208430DD10AE00843B0
:1027000004D000204FF0110B119072E7A3EB0B05E2
:102710006D1E0DE05B4504DD4FF0000205F1010583
:1027200004E003DA4FF00002A5F10105002AECD025
:1027300002981199C0E90231C0E9004579E700002B
:10274000000014400000F03F300000000000F043A3
:102750000000E03F2DE9FF4F95B09B4689460646B5
:1027600000250FE2252877D100242746F84A0121C9
:10277000059400E0044316F8013F203B01FA03F002
:102780001042F7D130782A2811D06FF02F0330781B
:10279000A0F13002092A16D8059A44F0020402EB8F
:1027A000820203EB42021044761C0590EFE759F8D1
:1027B000042B0592002A03DA504244F40054059099
:1027C00044F00204761C30782E2816D116F8010F3A
:1027D00044F004042A280DD06FF02F023078A0F1C5
:1027E0003003092B09D807EB870302EB4303C71813
:1027F000761CF3E759F8047B761C30786C280FD0F0
:1028000006DC4C2817D068280DD06A2814D104E0C3
:10281000742810D07A280FD10DE044F400140AE097
:1028200044F4801401E044F440147278824202D1EE
:1028300004F58014761C761C307866280BD013DCE7
:10284000582877D009DC002875D04528F6D04628CE
:10285000F4D047281AD19DE118E0632835D06428C8
:1028600079D0652812D195E1702873D008DC6728EB
:10287000F1D069286FD06E280DD06F2806D1B5E051
:1028800073282CD0752875D0782874D05A4617999B
:1028900090476D1C75E1C4F30250022809D003284B
:1028A0000DD0D9F8001004280DD00D6009F10409ED
:1028B00067E1D9F80010EA17C1E90052F6E7D9F844
:1028C00000100D80F2E70D70F0E719F8041B8DF889
:1028D000001000208DF80100EA46012003E059F8BD
:1028E00004AB4FF0FF3061074FF0000102D40DE060
:1028F00008F101018846B9420FDA8045F8DB1AF881
:1029000008100029F4D108E008F10101884681424D
:10291000FADB1AF808100029F6D105985B46A0EBFF
:10292000080721463846179A00F094FA284400EB2D
:10293000080507E04DE029E10DE01AF8010B5A46C1
:1029400017999047B8F10108F7D25B4621463846FF
:10295000179A13E142E00A220092C4F302524FF0A8
:10296000000A022A08D059F804CB032A4FEAEC7176
:102970000AD00DE029E02AE009F1070121F0070261
:10298000F2E802C1914609E00FFA8CFC4FEAEC71C3
:10299000042A03D14FFA8CFC4FEAEC71002907DAC4
:1029A0000A460021DCF1000C61EB02012D2202E05D
:1029B000220504D52B228DF80420012203E0E20732
:1029C00001D02022F7E7904659E00A2102E01022C8
:1029D0000DE010214FF0000A00910BE010224FF0A3
:1029E000000A44F004040827009203E008224FF094
:1029F000000A0092C4F30252022A05D059F804CB0F
:102A00000021032A08D009E009F1070121F007029B
:102A1000F2E802C1914605E01FFA8CFC042A01D1BC
:102A20000CF0FF0C4FF00008220728D5702806D0C4
:102A3000009B83F0100353EA0A0305D00EE0402206
:102A40008DF80420012208E05CEA010206D0302261
:102A50008DF804208DF8050002229046009B83F03B
:102A6000080353EA0A030AD15CEA010201D16207B2
:102A700005D530228DF804204FF001087F1E58281C
:102A800004D034A003900EA802900DE036A0F9E720
:102A900053466046009AFDF7ACFB84460398825C7F
:102AA0000298401E029002705CEA0100F0D1029888
:102AB00006A9081A00F1200A600702D524F4803420
:102AC00000E00127574502DDA7EB0A0000E00020E7
:102AD00000EB0A01009005984144401A0590E0037C
:102AE00006D45B462146179A059800F0B3F90544D1
:102AF000002706E001A85A46C05D179990476D1C53
:102B00007F1C4745F6DBE0030CD55B462146179A50
:102B1000059800F09FF9054404E030205A461799C3
:102B200090476D1C0099481E00900029F5DC08E0D4
:102B3000029802995A460078491C029117999047C9
:102B40006D1CBAF10001AAF1010AF1DC65E1000097
:102B50000928010030313233343536373839616273
:102B60006364656600000000303132333435363737
:102B700038394142434445460000000000F058F90E
:102B80000544761C307800287FF4ECAD19B0284657
:102B9000BDE8F08F620700D4062709F1070222F092
:102BA000070CFCE80223E14603F000485FEA080C4A
:102BB00002D00FF2702C0DE05FEA045C02D50FF238
:102BC000682C07E05FEAC47C02D00FF2602C01E0C1
:102BD000AFF2700C4FF0FF3823F00043CDF850C037
:102BE00065280CD006DC452809D046281DD047288A
:102BF0003DD13DE0662818D067287ED138E000211D
:102C0000112F01DB112000E0781CCDE9000106A99D
:102C10000EA8FFF7DDFCDDE90F010E9A03910021FC
:102C2000009207F1010A04914DE04FF00040009737
:102C3000CDE9011006A90EA8FFF7CAFCDDE90F02D5
:102C400003920E9B11990022DDF80CA000930492D0
:102C500011B9791C00EB010AB7EB0A0004D4C0F1EA
:102C6000FF3007F1010A0490AAEB0700019044E04D
:102C7000012F00DA01270021112F01DD112000E0D2
:102C80003846CDE9000106A90EA8FFF7A1FCDDE951
:102C90000F010E9A0391002104910092BA46210778
:102CA0000CD40399514500DA8A46BAF1010F05DDCB
:102CB000009AAAF10101515C302908D0B84202DA29
:102CC00010F1040F06DA0121CDE9011015E0AAF197
:102CD0000101E9E7002805DC049901440491AAEB0D
:102CE000000102E0411C514500DD8A460499401A6A
:102CF000401C01904FF000400290200704D401983E
:102D0000504501DBCDF8048000208DF84F0002987B
:102D10000DF14F07B0F1004F25D02B200E900298F7
:102D20004FF0020800280CDA404202902D200E904D
:102D300007E00A210298FDF746FA3031029007F8C1
:102D4000011DB8F10001A8F10108F2DC0298002889
:102D5000EFD1791E0E980870307800F0200040F016
:102D6000450007F8020D12A8C01B00F107081498CF
:102D7000007800B1012000EB0A01019801EBE0713D
:102D800005984144401A401E0590E00306D45B4676
:102D90002146179A059800F05DF8054414980078CC
:102DA00018B15A46179990476D1CE00324D55B462D
:102DB0002146179A059800F04DF805441CE0049848
:102DC000002807DBDDE90301884203DD0098405C51
:102DD000179901E0179930205A469047049805F159
:102DE0000105401C04900198401E019004D12E2042
:102DF0005A46179990476D1CBAF10001AAF1010AD1
:102E0000DDDC05E017F8010B5A46179990476D1C59
:102E1000B8F10001A8F10108F4DC5B462146179ADD
:102E20000598ABE62D0000002B00000020000000FC
:102E30002DE9F041044600251E461746880404D4B7
:102E400005E039462020B0476D1C641EF9D52846A0
:102E5000BDE8F0812DE9F041044600251E4690466C
:102E6000C80301D5302700E02027880404D505E0F9
:102E700041463846B0476D1C641EF9D52846BDE86A
:102E8000F0810A68531C0B601070704770B50446DF
:102E900000250948008800F4004058B10020064988
:102EA0000988C1F30E01054A505421461046FDF72A
:102EB00035F90546284670BD020000201025002087
:102EC0002DE9F04104460E4615460027002018491A
:102ED0000880FF2C07D800BF164800680028FBD1E7
:102EE00015490C8003E0214614A000F037F9DEB14B
:102EF000D5B112E00A2000F043F80D48008800F434
:102F0000004050B13046FFF7C1FF18B1002008491A
:102F1000088006E0002006490880681E80B2051E71
:102F2000E8D100BF05B901273846BDE8F0810000AF
:102F300002000020840002400444004025730D0A72
:102F40000000000010B504466FF00400FEF738FEE4
:102F5000E11704EB5171C1F3C701074A1170104624
:102F6000007800EB4001C1EBC0104FF6FF7101EAA1
:102F7000C0000249088010BD0400002006000020A7
:102F800001460D4A12884A434FF0E0235A6100225D
:102F90009A6101221A6100BF4FF0E022106900F02F
:102FA00001021AB100F48032002AF5D000224FF05D
:102FB000E0231A619A6170470600002070B504464C
:102FC0000D46E1B20548FFF7B6FA00BF0348008896
:102FD00000F080000028F9D0204670BD0038014084
:102FE00086B0504B0FCBCDE90423CDE9020100257B
:102FF0000024FEF7FBFD4820FFF7A4FFFEF7DCF8F6
:10300000FEF7FEF84FF48060FEF740F9FFF7ECF8AA
:10301000FEF7E8F944A0FFF795FA4FF47A70FFF74E
:10302000AFFF012010230222002100900846FEF786
:1030300079FB012010230322002100901846FEF79F
:1030400071FB012010233A22002100902020FEF77E
:10305000C9FAFDF779FC472140F2CF70FEF770FF07
:1030600041F61F41C720FEF71DFEFDF7BDFC58E0ED
:103070002F480078012832D100202D490870002205
:1030800001218807FFF715F8002201212948FFF7E1
:1030900010F8C820FFF774FF012211469007FFF7D0
:1030A00008F8012211462348FFF703F80121880799
:1030B000FEF7E2FF20480078012810D100201E49C9
:1030C00008701E480068282807DD1C480068A028F2
:1030D00003DA01251948047801E0002500241420B2
:1030E000FFF74EFF012D0AD10120102103232246B4
:1030F000CDE9001000212820FEF798FB07E0012011
:1031000010230FA2002100902020FEF7D9FB2046BB
:10311000FDF71DF80646FDF799FC21460BA0FFF7C9
:1031200011FAA5E7743200085374617274200A0022
:103130000800002000040040190000200C000020BE
:103140003A2D2D2D622F6D696E0000004865617269
:1031500074203D202564200D0A0D0A000FB438B5F7
:1031600005A800900B48009A0499FFF70FFA002079
:10317000009000BF084800680028FBD10548FCF714
:10318000DFFF84B221460448001FFFF71DF838BC5A
:103190005DF814FB10050020840002401CB50446B5
:1031A00001210420FEF70CFC01214804FEF7E8FB96
:1031B0002A48FFF7A5F80420ADF8000003208DF899
:1031C000020018208DF8030069462548FDF75BFFD3
:1031D0000820ADF8000048208DF80300694620481B
:1031E000FDF751FF1F48046000201E498880C880F9
:1031F000088188810C2048811848FFF72BF90122AB
:1032000080211648FFF772F8174A1449091D17481C
:10321000FEF7B6FF01211148FFF75CF8012240F2EA
:1032200025510E48FFF7F1F826208DF80400022002
:103230008DF8050003208DF8060001208DF80700A9
:1032400001A8FDF7EBFF41F61F416320FEF7CEFE1C
:10325000002007490880FEF7F5FE1CBD0044004031
:1032600000080140102900201005002080000240C5
:10327000020000202000000000000000000000000C
:10328000000000000000000000000000002F00000F
:1032900000000700070000147F147F1400242A7F19
:1032A0002A12006264081323003649552250000098
:1032B0000503000000001C224100000041221C0008
:1032C0000014083E08140008083E0808000000A08A
:1032D0006000000808080808000060600000002086
:1032E00010080402003E5149453E0000427F400064
:1032F000004261514946002141454B3100181412EA
:103300007F10002745454539003C4A4949300001B6
:103310007109050300364949493600064949291E05
:103320000000363600000000563600000008142267
:103330004100001414141414000041221408000267
:103340000151090600324959513E007C1211127C8C
:10335000007F49494936003E41414122007F4141B9
:10336000221C007F49494941007F09090901003EAB
:103370004149497A007F0808087F0000417F4100E9
:10338000002040413F01007F08142241007F40405F
:103390004040007F020C027F007F0408107F003E47
:1033A0004141413E007F09090906003E4151215E2D
:1033B000007F091929460046494949310001017F2A
:1033C0000101003F4040403F001F2040201F003FC0
:1033D0004038403F00631408146300070870080772
:1033E00000615149454300007F41410000552A5585
:1033F0002A55000041417F00000402010204004000
:103400004040404000000102040000205454547821
:10341000007F484444380038444444200038444441
:10342000487F00385454541800087E0901020018DF
:10343000A4A4A47C007F080404780000447D40001C
:10344000004080847D00007F102844000000417F00
:103450004000007C04180478007C080404780038DC
:103460004444443800FC242424180018242418FC64
:10347000007C0804040800485454542000043F44CD
:103480004020003C4040207C001C2040201C003C90
:103490004030403C004428102844001CA0A0A07CE0
:1034A000004464544C441414141414140000000018
:1034B00000000000000000000000FC000000000010
:1034C00002000000000C020C0200000000000000DE
:1034D00090D0BCD0BC900003000300001824FE4430
:1034E0008C000302070201001824D8B04C800003AE
:1034F00000010201C038E438E000010202010202CA
:10350000080600000000000000000000000000F8B5
:103510000402000000010204000204F8000000049C
:10352000020100009060F8609000000001000000BF
:103530002020FC202000000001000000000000000E
:1035400000000806000000002020202020000000CD
:103550000000000000000000000000020000000069
:103560000080601C0200040300000000F804040452
:10357000F8000102020201000008FC000000000245
:10358000030200001884442418000302020202000F
:1035900008042424D80001020202010040B088FC83
:1035A00080000000000302003C242424C400010227
:1035B00002020100F824242CC000010202020100D2
:1035C0000C04E41C0400000003000000D8242424A0
:1035D000D80001020202010038444444F80000030C
:1035E00002020100000010000000000002000000C4
:1035F00000002000000000000600000000205088AD
:1036000004020000000001029090909090000000E1
:1036100000000000000204885020000201000000A9
:103620001804C4241800000002000000F804E49408
:10363000F80001020202020000E09CF08000020398
:103640000000030204FC2424D8000203020201004B
:10365000F80404040C0001020202010004FC04044A
:10366000F80002030202010004FC24740C000203AF
:103670000202030004FC24740C0002030200000098
:10368000F0080444CC4000010202010004FC2020A8
:10369000FC040203000003020404FC040400020210
:1036A00003020200000404FC0404060404030000F6
:1036B00004FC24D00C0402030200030204FC0400F6
:1036C0000000020302020203FC3CC03CFC000300B9
:1036D0000300030004FC30C4FC04020302000300E6
:1036E000F8040404F80001020202010004FC24248E
:1036F0001800020302000000F8848404F8000102AC
:103700000207050004FC246498000203020003027F
:10371000182424448C000302020201000C04FC045F
:103720000C0000020302000004FC0000FC04000185
:1037300002020100047C80E01C0400000300000081
:103740001CE03CE01C00000300030000049C609CA3
:103750000400020300030200041CE01C0400000239
:10376000030200000C84641C040002030202030034
:103770000000FE020200000007040400000E30C03A
:103780000000000000010200000202FE0000000430
:103790000407000000040204000000000000000014
:1037A00000000000000008080808080800000200E7
:1037B00000000000000000000040A0A0C0000001C8
:1037C0000202030204FC2020C000000302020100E8
:1037D00000C02020600000010202020000C020247E
:1037E000FC0000010202030200C0A0A0C000000112
:1037F000020202000020F824240400020302020056
:103800000040A0A0602000070A0A0A0404FC20204F
:10381000C0000203020003020020E40000000002D6
:1038200003020000000020E4000008080807000070
:1038300004FC80E020200203020003020404FC00D8
:103840000000020203020200E020E020C0000300AA
:103850000300030020E02020C00002030200030256
:1038600000C02020C00000010202010020E0202052
:10387000C000080F0A02010000C02020E000000183
:10388000020A0F0820E0402020000203020000008E
:103890000060A0A020000002020203000020F82027
:1038A000000000000102020020E00020E000000112
:1038B0000202030220E020806020000003010000DB
:1038C0006080E080600000030003000020608060F2
:1038D000200002030003020020E02080602008088E
:1038E000070100000020A060200000020302020087
:1038F000000020DE0200000000070400000000FFBE
:1039000000000000000F00000002DE2000000004A4
:103910000700000002010204040200000000000091
:103920000000000000000000000000000000000097
:10393000000000F80000000000000033300000002C
:1039400000100C06100C0600000000000000000033
:1039500040C07840C0784000043F04043F040400A5
:10396000007088FC08300000001820FF211E0000B5
:10397000F008F000E018000000211C031E211E00CA
:1039800000F00888700000001E2123241927211050
:1039900010160E00000000000000000000000000F3
:1039A000000000E01804020000000007182040009A
:1039B00000020418E000000000402018070000008A
:1039C000404080F0804040000202010F01020200EE
:1039D000000000F0000000000101011F01010100D2
:1039E000000000000000000080B070000000000037
:1039F00000000000000000000001010101010101C0
:103A00000000000000000000003030000000000056
:103A1000000000008060180400601806010000002B
:103A200000E010080810E000000F102020100F0028
:103A3000001010F8000000000020203F20200000AF
:103A40000070080808887000003028242221300007
:103A500000300888884830000018202020110E000F
:103A60000000C02010F8000000070424243F2400B8
:103A700000F80888880808000019212020110E008D
:103A800000E0108888180000000F112020110E009F
:103A900000380808C83808000000003F0000000097
:103AA0000070880808887000001C222121221C0058
:103AB00000E010080810E0000000312222110F0081
:103AC000000000C0C0000000000000303000000016
:103AD0000000008000000000000080600000000086
:103AE000000080402010080000010204081020009F
:103AF00040404040404040000404040404040400EA
:103B0000000810204080000000201008040201007E
:103B1000007048080808F00000000030360100007E
:103B2000C030C828E810E0000718272423140B0031
:103B30000000C038E0000000203C230202273820AB
:103B400008F8888888700000203F202020110E008F
:103B5000C030080808083800071820202010080086
:103B600008F808080810E000203F202020100F006F
:103B700008F88888E8081000203F2020232018003B
:103B800008F88888E8081000203F200003000000A3
:103B9000C03008080838000007182020221E020044
:103BA00008F808000008F808203F210101213F2003
:103BB000000808F8080800000020203F202000002E
:103BC00000000808F8080800C08080807F0000001E
:103BD00008F888C028180800203F20012638200057
:103BE00008F8080000000000203F202020203000BE
:103BF00008F8F800F8F80800203F003F003F2000D8
:103C000008F830C00008F808203F200007183F00DF
:103C1000E01008080810E0000F10202020100F000E
:103C200008F808080808F000203F21010101000001
:103C3000E01008080810E0000F18242438504F0046
:103C400008F8888888887000203F2000030C302006
:103C500000708808080838000038202121221C0044
:103C6000180808F8080818000000203F200000008D
:103C700008F808000008F808001F202020201F0076
:103C80000878880000C83808000007380E010000D6
:103C9000F80800F80008F800033C0700073C0300A0
:103CA000081868808068180820302C03032C302006
:103CB0000838C800C83808000000203F2000000075
:103CC00010080808C83808002038262120201800CD
:103CD000000000FE020202000000007F40404000A1
:103CE000000C30C000000000000000010638C000D9
:103CF00000020202FE000000004040407F00000081
:103D000000000402020204000000000000000000A5
:103D100000000000000000008080808080808080A3
:103D2000000202040000000000000000000000008B
:103D300000008080808000000019242222223F2081
:103D400008F8008080000000003F112020110E00C4
:103D50000000008080800000000E11202020110053
:103D6000000000808088F800000E112020103F2005
:103D70000000808080800000001F22222222130089
:103D8000008080F0888888180020203F20200000D4
:103D90000000808080808000006B94949493600089
:103DA00008F8008080800000203F210000203F2094
:103DB00000809898000000000020203F2020000094
:103DC000000000809898000000C08080807F000084
:103DD00008F8000080808000203F24022D30200061
:103DE000000808F8000000000020203F202000000C
:103DF0008080808080808000203F20003F20003F26
:103E00008080008080800000203F210000203F2033
:103E10000000808080800000001F202020201F00E4
:103E2000808000808000000080FFA12020110E0013
:103E30000000008080808000000E112020A0FF8004
:103E4000808080008080800020203F2120000100B1
:103E50000000808080808000003324242424190006
:103E6000008080E0808000000000001F2020000013
:103E70008080000000808000001F202020103F2054
:103E8000808080000080808000010E3008060100E4
:103E900080800080008080800F300C030C300F0089
:103EA00000808000808080000020312E0E312000B4
:103EB000808080000080808080818E7018060100E4
:103EC00000808080808080000021302C2221300002
:103ED00000000000807C020200000000003F404023
:103EE00000000000FF00000000000000FF000000D4
:103EF0000002027C800000000040403F0000000003
:103F0000000601010202040400000000000000009D
:103F100000000000000000000000000000000000A1
:103F20000000000000000000000000000000000091
:103F3000000000000000000000F0F0F000000000B1
:103F40000000000000017F010000000000000000F0
:103F5000001C1C1C0000000000008060301C8C60F5
:103F6000301C0C00000000000000000000000000F9
:103F7000000000000000000000000000000000E061
:103F80000000000000E000000086E69F868686862E
:103F9000E69F860000011F01010101011F010100D0
:103FA000000080C06020F820E0C00000000003078F
:103FB0000C18FF70E18100000000070F10107F1047
:103FC0000F0700008060206080000000E0200000FB
:103FD0000F3020309F70DC371030C0000000100E12
:103FE00003000718101807000000C02020E0C000E0
:103FF0000000000080E01F38E88703C43C04000094
:10400000070F1810100B070D1010080000808C4CC3
:104010003800000000000000000000000000000068
:104020000000000000000000000000000000000090
:1040300000000000000080E03008040000000000E4
:1040400000FEFF0100000000000000000000030F60
:104050001820400000040830E0800000000000004C
:104060000000000001FFFE000000000000402018DA
:104070000F03000000000000000000000000C0006E
:1040800000000000004266663C18FF183C6666426D
:10409000000000000000030000000000000000001D
:1040A0000000800000000000001010101010FF1031
:1040B00010101010000000000000030000000000BD
:1040C00000000000000000000000000000000000F0
:1040D000000000000000000000808C4C3800000050
:1040E00000000000000000000000000000000000D0
:1040F0000010101010101010101010000000000020
:1041000000000000000000000000000000000000AF
:10411000000000000000000000000000000000009F
:1041200000001C1C1C00000000000000000000003B
:1041300000000000E0380C000000000080701C034C
:10414000000000000060380E0100000000000000C8
:10415000000080C060202060C080000000FEFF01E1
:104160000000000001FFFE000001070E18101018EB
:104170000E0701000000808080C0E0000000000009
:104180000000000000FFFF00000000000000101011
:10419000101F1F1010100000008040202020206001
:1041A000C080000000030300804020381F0700008B
:1041B000001C1A1918181818181F00000080C020B9
:1041C000202060C080000000000303001010182FA2
:1041D000E780000000070F10101010180F070000F4
:1041E000000000000000C0E0F000000000C0B08847
:1041F000868180FFFF808000000000000010101FFB
:104200001F1010000000E0606060606060600000EF
:1042100000003F1008080818F0E0000000070B102D
:104220001010101C0F030000000080C04020202050
:10423000E0C0000000FCFF211008080818F0E000B2
:104240000001070C18101010080F03000000C0E058
:104250006060606060E06000000003000000E01843
:104260000700000000000000001F1F000000000009
:104270000080C0602020202060C080000087EF2CDC
:104280001818303068CF830000070F081010101086
:10429000180F07000000C0C020202020C0800000B0
:1042A000001F3F604040402010FFFE0000000C1C3B
:1042B000101010080F0300000000000000000000B4
:1042C0000000000000000000000E0E0E00000000C4
:1042D00000000000001C1C1C00000000000000008A
:1042E000000000000000000000000000000C0C00B6
:1042F000000000000000000000583800000000002E
:104300000000000000000080402010000000102885
:1043100044820100000000000000000000000102D3
:104320000408100000000000000000000000000071
:104330000084848484848484848484000000000055
:10434000000000000000000000001020408000007D
:10435000000000000000000000000182442810005E
:1043600000001008040201000000000000C020202E
:104370001010101030E0C0000003030000F010081F
:104380000C070300000000001C1C1C0000000000C3
:10439000000000C0406020202040C00000FCFF0161
:1043A000F00E03C1FE03807F0001070E08111110FB
:1043B000110904020000000080E0E000000000009D
:1043C0000000807C4340477FF880000010181F10D9
:1043D00000000000131F1C1020E0E02020202060BF
:1043E000C080000000FFFF10101010182FE78000A1
:1043F000101F1F1010101010180F0700000080C0B1
:10440000402020202060E00000FCFF0100000000B0
:10441000000001000001070E18101010080403002E
:1044200020E0E02020202040C080000000FFFF00AE
:104430000000000001FFFE00101F1F1010101808E0
:104440000E07010020E0E0202020202020608000D6
:1044500000FFFF101010107C00000000101F1F1044
:10446000101010101018060020E0E020202020205E
:104470006060800000FFFF101010107C0000010041
:10448000101F1F100000000000000000000080C08E
:104490006020202040E0000000FCFF0100004040C0
:1044A000C0C140400001070E181010100F0F00008F
:1044B00020E0E0200000000020E0E02000FFFF10EE
:1044C0001010101010FFFF00101F1F100000000040
:1044D000101F1F100000202020E0E02020200000FE
:1044E0000000000000FFFF000000000000001010AE
:1044F000101F1F101010000000000000202020E0FE
:10450000E020202000000000000000FFFF0000006D
:104510000060E0808080C07F3F00000020E0E0205D
:10452000000020A06020200000FFFF30187CE3C0C6
:1045300000000000101F1F10000001131F1C1810A6
:1045400020E0E020000000000000000000FFFF006D
:104550000000000000000000101F1F1010101010BD
:104560001018060020E0E0E000000000E0E0E0209D
:1045700000FF013FFEC0E01E01FFFF00101F100002
:10458000031F0300101F1F1020E0E0C00000000008
:104590000020E02000FF0003071C78E08000FF00FF
:1045A000101F100000000000030F1F00000080C05B
:1045B00060202060C080000000FEFF0100000000BD
:1045C00000FFFE000001070E181010180C07010074
:1045D00020E0E0202020202060C0800000FFFF209D
:1045E00020202020301F0F00101F1F10000000008F
:1045F00000000000000080C060202060C08000003B
:1046000000FEFF010000000000FFFE000001070E99
:104610001111133C7C67210020E0E02020202020A5
:1046200060C0800000FFFF101030F0D0080F0700BE
:10463000101F1F10000000030F1C10100080C0602E
:10464000202020204040E00000070F0C18183030D8
:1046500060E08100001F0C0810101010180F0700F8
:104660008060202020E0E020202060800100000009
:1046700000FFFF000000000100000000101F1F10DD
:104680000000000020E0E020000000000020E0200A
:1046900000FFFF00000000000000FF0000070F18EF
:1046A00010101010100807002060E0E0200000004B
:1046B00020E060200000077FF88000807C0300007D
:1046C00000000000071F1C070000000020E0E020A1
:1046D00000E0E0200020E0200007FFF8E01FFFFCE2
:1046E000E01F00000000031F0300011F0300000083
:1046F000002060E0A0000020E06020000000000337
:104700008F7CF8C6010000000010181E130001176E
:104710001F1810002060E0E02000000020E0602072
:10472000000001073EF8E01807000000000000103C
:10473000101F1F101000000000806020202020A00B
:10474000E0E0200000000000C0F03E0F0300000089
:1047500000101C1F17101010101806000000000099
:1047600000FC0404040404000000000000FF00003A
:104770000000000000000000007F4040404040007A
:10478000000010E000000000000000000000000039
:10479000031C608000000000000000000000000317
:1047A0000C70800000000404040404FC00000000FD
:1047B00000000000000000FF00000000000040407A
:1047C0004040407F0000000000000010080C040C76
:1047D00008100000000000000000000000000000C1
:1047E00000000000000000000000000000000000C9
:1047F00000000000000000000000000000000000B9
:1048000000000000808080808080808080808080A8
:104810000000000404080800000000000000000080
:104820000000000000000000000000000000000088
:104830000000000000000000000000000000000078
:10484000000098D844642424FCF80000000F1F18CE
:10485000101010081F1F10180020E0F000000000CA
:10486000000000000000FFFF180804040CF8F0002E
:1048700000001F0F18101010180F03000000000098
:10488000000000000000000000E0F8180404043CF0
:104890003800000000030F0C101010100806000074
:1048A0000000000000000020E0F0000000E0F81C24
:1048B00004040408FFFF000000030F181010100884
:1048C0001F0F0800000000000000000000000000B2
:1048D0000000E0F8484444444C7870000000030FA6
:1048E0000C181010100804000000000080C06020A8
:1048F00020E0C00000040404FFFF040404040000DE
:10490000000010101F1F1010100000000000000019
:104910000000000000000000000070F88C04048C0F
:10492000F874040C007076CF8D8D8D89C878700076
:104930000020E0F000000000000000000000FFFF89
:1049400008040404FCF8000000101F1F10000010F1
:104950001F1F100000000000006060000000000049
:104960000000040404FCFC00000000000000101023
:10497000101F1F1010100000000000000000006059
:104980006000000000000000040404FCFC000000C3
:104990000000C0C08080C07F3F0000000020E0F029
:1049A00000000000000000000000FFFF80C0F41CB9
:1049B0000404000000101F1F1100031F1C10100032
:1049C0000000202020E0F0000000000000000000B7
:1049D00000FFFF000000000000001010101F1F105B
:1049E00010100000000000000000000000000000A7
:1049F00004FCFC0804FCFC0804FCFC00101F1F1055
:104A0000001F1F10001F1F1000000000000000000A
:104A1000000000000004FCFC08080404FCF800008E
:104A200000101F1F100000101F1F100000000000CA
:104A3000000000000000000000E0F0180C04040C6E
:104A400018F0E00000030F0C101010100C0F030002
:104A50000000000000000000000000000004FCFC5A
:104A6000080404040CF8F0000080FFFF8890101088
:104A70001C0F030000000000000000000000000008
:104A800000E0F81C04040408F8FC000000030F1800
:104A900010109088FFFF8000000000000000000060
:104AA00000000000040404FCFC100804040C0C00CA
:104AB0001010101F1F101010000000000000000058
:104AC000000000000000000000003078CCC48484A6
:104AD000840C1C0000001E1810101011190F060085
:104AE0000000000000C000000000000000040404FA
:104AF000FFFF040404000000000000000F1F10105E
:104B0000100C000000000000000000000000000089
:104B10000004FCFE00000004FCFE000000000F1F6B
:104B2000181010081F0F080000000000000000000F
:104B30000000000000040C3CFCC40000C43C0C0459
:104B400000000000010F1E0E010000000000000028
:104B50000000000000000000043CFCC400E47CFCF9
:104B600084807C040000071F070000071F07000067
:104B70000000000000000000000000000004041C11
:104B80007CE4C0341C0404000010101C1601131F28
:104B90001C181000000000000000000000000000D1
:104BA00000040C3CFCC400C43C0404000000C080B1
:104BB000C1370E01000000000000000000000000EE
:104BC0000000000000001C0404C4F47C1C0400006D
:104BD0000000101C1F17111010180E00000000001C
:104BE000000000F80C04000000000000001028EF96
:104BF00000000000000000000000003F60400000D6
:104C0000000000000000FF000000000000000000A5
:104C10000000FF0000000000000000000000FF0096
:104C2000000000000000040CF8000000000000007C
:104C300000000000EF2810000000000000004060AD
:104C40003F000000000000000018060202040810E7
:104C500020203008000000000000000000000000DC
:104C60000000000000000000000000000000F80844
:104C700008F80C0B08F80808F800000040407F40D6
:104C8000407F4040407F40407F40400000000000A7
:104C90000000000000000000000000000000000014
:104CA0000000000000000000000000000824236A4B
:104CB000AA2AAA6A2A2A2AEA020200001011151555
:104CC00015FF15151511100F3040F80000000000F9
:104CD00000000000000000000000000000000000D4
:104CE0000000000000000000000000000000008044
:104CF0000000E002041800000040800000100C03D7
:104D000000003F40404040407800010E000000009D
:104D10000000000000000000000000000000000093
:104D2000000000000000000000000000000014A4CB
:104D3000442434AD6624940444A4140000080908F3
:104D400008090909FD09090B080809080000000005
:104D50000000000000000000000000000000000053
:104D6000000000000000000000000000000000C083
:104D700080808080808080FC84808080808080C073
:104D8000C0000000000000FF7F404040404040FF66
:104D900040404040404040FF7F00000000000000D5
:104DA000000000000000007F700000000000000014
:104DB00000000000000000000000000000000000F3
:104DC000000000FCF80000000000000000000000EF
:104DD0000000000000000000FFFE020202020202CA
:104DE000020202FFFF020202020202020202FF03AB
:104DF00000000000000000001F1F0404040404045D
:104E0000040404FFFF0404040404040404041F0055
:104E10000000000000000000000000000000000092
:104E20000000007F3F0000000000000000000000C4
:104E30000000000000000000000000000000000072
:104E40000000000000000000000000000000000062
:104E500000F8F8F0F07020000000000000000000F2
:104E60000000000000000000000000000000000042
:104E700000000000000000000000000080000000B2
:104E80000000000000000000000000000000000022
:104E900000FFFFFFFF000000000000000000000016
:104EA0000000000000000000808000000000000002
:104EB00000000000000000000000000000FFFFFEF6
:104EC0000606060606060606060606060606060682
:104ED00006FFFFFFFF06060606060606060606068E
:104EE00006060606060606FFFFFFFF070200000093
:104EF00000000000000000000000000000FFFFFFB5
:104F000000000000000000000000000000000000A1
:104F100000FFFFFFFF000000000000000000000095
:104F200000000000000000FFFFFFFF000000000085
:104F300000000000000000000000000000FFFFFF74
:104F400018181818181818181818181818181818E1
:104F500018FFFFFFFF181818181818181818181835
:104F600018181818181818FFFFFFFF00000000009D
:104F7000000000000000000000000000020101002D
:104F80000000000000000000000000000000000021
:104F900000FFFFFFFF000000000000000000000015
:104FA00000000000000000010100000000000000FF
:104FB00000000000000000000000000000000000F1
:104FC00000000000000000000000000000000000E1
:104FD00000FFFFFFFF0000000000000000000000D5
:104FE00000000000000000000000000000000000C1
:104FF00000000000000000000000000000000000B1
:1050000000000000000000000000000000000000A0
:10501000001F1F0F0F000000000000000000000034
:105020000000000000000000000000000000000080
:10503000000000005450000800000020580000004C
:10504000B0250008AC50000858000020F02A0000ED
:10505000C025000800000000000000000000000063
:1050600000000000000000005802000000000000E6
:10507000000000000000000000020000000200002C
:1050800000020000640000000000000001000000B9
:1050900000000000000000000102030401020304FC
:0C50A000060708090204060800000000D2
:04000005080000ED02
:00000001FF
